:020000000A28CC
:10000800FE00030EF0000A08F100D62AF02AB40117
:10001800B501AF01AA014008B8003F08B700DF30BA
:10002800BA01BB01BC01BD01B001B101B201B3010C
:10003800AD01AE01AB01AC018316810064008B01F8
:10004800FD30831603138500831285013F30831624
:10005800860083128601FF30A801B601A901F900C4
:10006800AE22FF30F200F300E422F901AE22FF30A5
:10007800F200F300E422FF30F900AE22FF30F20074
:10008800F300E422F90183120313B901B90AF9173D
:1000980001302022F7007719562820302022F70057
:1000A800F71C5828B901F913AE2211300B11810041
:1000B800A0308B007818E02837080319DF28B90822
:1000C800031DBF2801302022BE003E1BBE1E712822
:1000D8003E1E71280430BE008628BE183E1E8628A3
:1000E8001030F201F20A8422003A03197D28023006
:1000F80085280130F201F20A8422003A03197B288C
:100108001030BE063E08463903199028B401BA01DA
:10011800BB01B001B101DF283E1EA3280430B401A1
:10012800BA070318BB0A00303B028C3003193A02A5
:10013800031CDF28BA01BB01B001B101DA28043081
:10014800B0070318B10A003031028C3003193002AD
:10015800031CDF28BA01BB01B001B101AF01AF0A2E
:10016800B7017916791BBC28B408031DBC28791778
:10017800B401B40ADF28390BDF2808302022BE007A
:100188003E1CCA283E0842390319CD28BA01BB01D2
:10019800DF280430BA070318BB0A00303B023230AC
:1001A80003193A02031CDF28BA01BB01AF01AF0AE9
:1001B800B701F9157917AE22F81CE028F81078185D
:1001C8006229380803196129B908031D412920301B
:1001D8002022BE003E1B3E1CF528BE1DF52802301D
:1001E800BE003E19BE1D08290830F2018422003ADB
:1001F80003190029043007292030F2018422003A2B
:100208000319FE280830BE063E084639031912298C
:10021800B501BC01BD01B201B3016129BE1D25298B
:100228000430B501BC070318BD0A00303D028C300C
:1002380003193C02031C6129BC01BD01B201B301D1
:100248005C290430B2070318B30A003033028C303B
:1002580003193202031C6129BC01BD01B201B301BB
:10026800AF01AF0AB8017914791B3E29B508031DFF
:100278003E297917B501B50A6129390B6129103072
:100288002022BE00BE1E4C293E08443903194F29BE
:10029800BC01BD0161290430BC070318BD0A003048
:1002A8003D02323003193C02031C6129BC01BD0127
:1002B800AF01AF0AB80179157917AE22F81C622987
:1002C800F810051E6D297818812978147913AE2243
:1002D8008129781C8129F911791179127910AA01DB
:1002E800AF01AD01AE01AB01AC01B701B70AB8016E
:1002F800B80AB401B501AE2278107818A729F91206
:10030800F910B908031D97290830F2015A22003A5A
:10031800031DF9161030F201F20A5A22003A0319A5
:10032800A629F914A629390BA6290930F2015A225F
:10033800003A031DF9163030F201F20A5A22003A47
:10034800031D9529AE22F81CA729F8107818ED2965
:100358002A080319CD290430AB070318AC0A4E301C
:100368002C02203003192B02031879134E302C026B
:10037800203003192B02031CCD29F91179117912A8
:1003880079107913AA01AB01AC01B701B70AB8011A
:10039800B80A2F080319ED290430AD070318AE0A6F
:1003A800B908031DE6290B302E02B83003192D02B7
:1003B800031CED29AD01AE01AF01AA01AA0AB701DC
:1003C800B801ED2901302E02C23003192D0203189D
:1003D800DE292908A7003608A9000508B60001305B
:1003E800B60536082906031D1B2A36082706031DED
:1003F8001B2A3608280603191B2A36080319192A46
:10040800F901390B092AB9010C2AB901B90AF917F6
:10041800AA01AF01AD01AE01AB01AC01B701B70A4A
:10042800B801B80AB401B50178103608A800AE22A0
:10043800F81C1C2AF8105E28A300393A8316860097
:100448008312230886000F30A400A40B292A05086C
:10045800A6002C30A6050608A5003930A5050F30E2
:10046800A400A40B352A0508A1002C30A105060814
:10047800A2003930A20526082106031D272A2508CF
:100488002206031D272A3930831686008312860127
:100498002608F20006300310F20C7205F300031070
:1004A800260D403973042504A0000800F5000A3021
:1004B8009F00873083169F007508393C86007508B1
:1004C800831286000F30F600F60B682A4030F300DE
:1004D800720A702A0310F30DFF3E031D6E2A73087B
:1004E8001F050319792AF4017B2AF401F40A0F3055
:1004F8009F0039308316860083128601740808002D
:10050800F5000A309F008E3083169F007508393A2F
:1005180086007508831286000F30F600F60B922AC3
:100528004030F300720A9A2A0310F30DFF3E031DB0
:10053800982A73081F050319A32AF401A52AF401B0
:10054800F40A0F309F003930831686008312860123
:100558007408080079082D390319B72A0230831264
:1005680003138500BA2A8312031385018030F20031
:10057800F301F401790872050319C42A4030F40024
:10058800740886007408803886007408860008306D
:100598000310F20CF30A7302031CBD2A0230860012
:1005A8008601080011308312031381006400F814D7
:1005B8000B1171088A00700E8300FE0E7E0E090072
:1005C800730800380319080064000130F202003093
:1005D800031CF303F302E42A0130F801BF00C00052
:0405E80083010B2858
:02400E000E3F63
:00000001FF
